:020000040800F2
:1040000000C0002025650008F9620008FB62000876
:10401000FD620008FF620008016300080000000064
:104020000000000000000000000000000363000822
:10403000056300080000000007630008096300082A
:104040006D6500086D6500086D6500086D65000808
:104050006D6500086D6500086D6500086D650008F8
:104060006D6500086D6500086D6500086D650008E8
:104070006D6500086D6500080D6300081963000890
:1040800025630008316300083D6300086D65000882
:104090006D6500086D6500086D6500086D650008B8
:1040A0006D6500086D6500086D6500086D650008A8
:1040B0006D6500086D6500086D6500086D65000898
:1040C0006D6500086D6500086D6500086D65000888
:1040D0006D65000859630008656300086D65000898
:1040E0006D6500086D6500086D6500086D65000868
:1040F0006D6500086D6500086D6500087163000856
:104100006D6500086D6500086D6500086D65000847
:104110007D6300086D650008896300086D6500080F
:104120006D6500086D6500086D6500086D65000827
:10413000000000000000000000000000000000007F
:10414000000000000000000000000000000000006F
:10415000000000000000000000000000000000005F
:10416000000000000000000000000000000000004F
:10417000000000000000000000000000000000003F
:10418000000000000000000000000000000000002F
:10419000000000000000000000000000000000001F
:1041A000000000000000000000000000000000000F
:1041B00000000000000000000000000000000000FF
:1041C00000000000000000000000000000000000EF
:1041D00000000000000000000000000000000000DF
:0441E0005FF8E0F1B3
:1041E40010B5054C237833B9044B13B10448AFF32D
:1041F40000800123237010BD700200200000000025
:10420400B476000808B5034B1BB103490348AFF368
:10421400008008BD0000000074020020B47600088D
:1042240038B50E4B054618784FF47A73B3FBF0F3A8
:104234000B4A1068B0FBF3F000F04AFA044658B990
:104244000F2D09D8024629464FF0FF3000F0FEF941
:10425400044B20461D6038BD012038BD00000020FD
:104264000802002004000020074A08B51368032050
:1042740043F01003136000F0D7F90020FFF7D0FFDC
:1042840001F0B2FE002008BD00200240034A044BA6
:1042940011681B780B441360704700BFA80200200C
:1042A40000000020014B1868704700BFA8020020DE
:1042B40038B50446FFF7F6FF0546631C1EBF044BE2
:1042C4001B78E418FFF7EEFF401B8442FAD838BD90
:1042D4000000002070477047036810B55A68044610
:1042E400900627D51A68910724D5A26AD2065EBF24
:1042F400A26A42F40072A2629A6802F46022B2F5E1
:10430400602F10D1227B72B95A6822F020025A60C1
:10431400A36A23F48073A362A36ADB045EBFA36A67
:1043240043F00103A3622046FFF7D4FF6FF01202AB
:1043340023681A6023685A68100630D51A68510732
:104344002DD5A26AD2065EBFA26A42F40052A262CE
:104354009A6802F4E042B2F5E04F0AD05A68500578
:1043640016D49A6802F46022B2F5602F10D1227B31
:1043740072B95A6822F080025A60A36A23F4805307
:10438400A362A36AD9055EBFA36A43F00103A362D3
:10439400204600F047F96FF00C0223681A60236886
:1043A4005A6852060DD51B68DB070AD5A36A204656
:1043B40043F48033A362FFF78EFF6FF0010223689A
:1043C4001A6010BD002373B5019390F82430012BBB
:1043D40074D001234D6880F82430062D02684FEA1A
:1043E40085030C6825D82B441F25566B053B9D403F
:1043F40026EA050504FA03F32B435363092C4FEA19
:1044040044038D682FD907262344D1681E3B9E4060
:1044140021EA060105FA03F30B43D360A4F1100368
:10442400012B2BD90023002280F82420184602B047
:1044340070BD0C2D0BD82B441F25166B233B9D40C0
:1044440026EA050504FA03F32B431363D6E72B444A
:104454001F25D66A413B9D4026EA050504FA03F36D
:104464002B43D362CAE70726116923449E4021EAFD
:10447400060105FA03F30B431361CFE7104B9A428D
:1044840016D193681B02CDD49368102C43F4000317
:104494009360C7D10B4B0C4A1B68B3FBF2F20A239F
:1044A40053430193019B002BBCD0019B013BF8E7D4
:1044B400836A43F0200383620123B4E70223B5E750
:1044C400002401400802002040420F0038B5036870
:1044D40004469A68D20701D4002038BD9A6822F0B5
:1044E40001029A60FFF7DEFE054623689B68DB073E
:1044F400F2D5FFF7D7FE401B0228F6D9A36A0120A4
:1045040043F01003A362E36A43F00103E36238BD9E
:10451400F8B50446002877D0836A23B9C36280F8CB
:10452400243001F083FD2046FFF7D0FFA36A13F087
:1045340010036BD1002869D1A26A374922F488524A
:1045440022F0020242F00202A26294E824008A42AB
:10455400E16904D1B1F5402F08BF4FF40021267B57
:1045640045EA46052943A568B5F5807F35D0012D78
:1045740008BF4FF48073277D012F06D17EBBA66947
:10458400013E43EA463343F400635668B5F5807F41
:1045940026F4694643EA0603536096681F4B03EA10
:1045A400060343EA0103936001D0012D20D123695E
:1045B400013B1B05D56A25F470052B43D362926831
:1045C400174B1340994215D10023E362A36A23F0E9
:1045D400030343F00103A362F8BD2B46CBE7A66AAD
:1045E40046F02006A662E66A46F00106E662CCE7DB
:1045F4000023DFE7A36A23F0120343F01003A3624E
:10460400E36A43F00103E3620120F8BDA36A43F0C7
:104614001003A362F8E700BF003C0140FDF7E1FF8F
:10462400FE0E1FFF70470000074A0002D36800F423
:10463400E06023F4E0631B041B0C43F0BF6343F40A
:1046440000330343D360704700ED00E0174B30B5EF
:10465400DC68C4F30224C4F10703251D042B28BF1E
:104664000423062D4FF0010598BF002405FA03F337
:1046740003F1FF3388BF033C1940A14005FA04F459
:10468400013C2240002842EA01024FEA0212A9BF7B
:1046940000F16040064BD2B200F56140BBBF00F0B0
:1046A4000F00D2B280F800231A5430BD00ED00E0B0
:1046B40014ED00E0002808DB0123420900F01F008C
:1046C40003FA00F0014B43F82200704700E100E0D8
:1046D4000138B0F1807F0AD2F021064B064A5860B7
:1046E40082F823100020072298601A607047012086
:1046F400704700BF10E000E000ED00E010B50028B6
:1047040032D00168194B1424994225D8184AA3F2CF
:1047140007430A44B2FBF4F2920002648468C36360
:1047240043680A682343C46822F47F52234304691C
:1047340022F0300223434469234384692343C46938
:10474400234313430B600122002380F82120836359
:1047540080F82030184610BD064B0B44B3FBF4F32D
:104764009B000364044BD9E7012010BD07040240F9
:10477400F8FFFDBFF8FBFDBF00040240F0B590F860
:104784002040012C35D0012490F8215080F820409D
:10479400A5424FF000064FF0020428D180F82140D2
:1047A400046886632668076C26F001062660C66BDB
:1047B400BD407560636043680568102BC36A0BBF16
:1047C400A260A160E160E2604BB1236843F00E0394
:1047D40023602B68002043F001032B60F0BD2368A5
:1047E40023F004032360236843F00A03F0E780F80E
:1047F40020600220F0BD000090F8213010B5022B9B
:1048040003D004238363012010BD03681A6822F0D7
:104814000E021A601A6822F001021A60294A9342B1
:1048240024D902F56272934219D01432934218D0FB
:104834001432934217D0143293420CBF4FF4805376
:104844004FF48033204A53600123002480F8213040
:10485400436B80F820409BB39847204610BD01234A
:10486400F0E71023EEE74FF48073EBE717498B4230
:1048740016D014318B4215D014318B4214D014311C
:104884008B4214D014318B4214D014318B4214D087
:10489400934214BF4FF480334FF080730C4AD2E735
:1048A4000123FBE71023F9E74FF48073F6E74FF495
:1048B4008053F3E74FF48033F0E74FF48013EDE7D0
:1048C400184610BD80000240000402400800024067
:1048D4000000024070B40425C66B026C346803689F
:1048E40095402542196855D04D0753D51A68960648
:1048F4005EBF1A6822F004021A60604A93421FD90C
:1049040002F56272934214D01432934213D01432DB
:10491400934212D0143293420CBF4FF480434FF4AD
:104924008023574A5360C36A002B00F0A58070BCF3
:1049340018470423F5E74023F3E74FF48063F0E7D7
:1049440050498B4216D014318B4215D014318B420E
:1049540014D014318B4214D014318B4214D014313E
:104964008B4214D0934214BF4FF480234FF08063E2
:10497400454AD7E70423FBE74023F9E74FF4806374
:10498400F6E74FF48043F3E74FF48023F0E74FF466
:104994008003EDE702259540254257D08D0755D574
:1049A4001A68940606D41A6822F00A021A600122D0
:1049B40080F82120314A93421ED902F56272934253
:1049C40013D01432934212D01432934211D01432C1
:1049D40093420CBF4FF400534FF40033284A536002
:1049E400002380F82030836A9EE70223F6E7202321
:1049F400F4E74FF40073F1E722498B4216D01431E7
:104A04008B4215D014318B4214D014318B4214D004
:104A140014318B4214D014318B4214D0934214BFFE
:104A24004FF400334FF00073174AD8E70223FBE733
:104A34002023F9E74FF40073F6E74FF40053F3E74C
:104A44004FF40033F0E74FF40013EDE708259540E9
:104A5400254211D009070FD5196821F00E011960FC
:104A6400012303FA02F27260836380F82130002389
:104A740080F82030036B57E770BC70478000024019
:104A84000004024008000240000002402DE9F74FF4
:104A9400002426466C4F6D4BDFF8B8E1DFF8B8C14F
:104AA4000A6832FA06F502D103B0BDE8F08F4FF080
:104AB400010808FA06F802EA0802904540F08480EA
:104AC4004D68122D00F0B18000F28780022D00F0B5
:104AD400A9807BD8002D00F08C80012D00F0A080EF
:104AE4004FF00F09FF2A93BF824606F18045083D27
:104AF400D0F800B092BFB500D0F804B0AD0009FA08
:104B040005F82BEA080804FA05F588BF00F1040A41
:104B140048EA0505CAF80050D1F804A01AF0805FED
:104B240052D0BD6926F0030845F00105BD61BD6999
:104B340008F1804805F00105019508F5803806F074
:104B4400030B019D4FEA8B0BD8F8085009FA0BF9B7
:104B540025EA09093E4DA8426CD005F58065A842B6
:104B64006AD005F58065A84268D005F58065A8423D
:104B740066D005F58065A84264D070450CBF052554
:104B8400062505FA0BF545EA0905C8F808501D681D
:104B94001AF4803F14BF154395431D605D681AF4F1
:104BA400003F14BF154395435D609D681AF4801F50
:104BB40014BF154395439D60DD681AF4001F14BFAC
:104BC4002A4325EA0202DA60013669E7032D25D07B
:104BD400112D85D1CC68043482E7654509D012D8FB
:104BE400DFF878904D4504D009F580394D457FF4C0
:104BF40077AF8C68E4B1012C0CBFC0F81080C0F80A
:104C0400148008246CE7DFF858904D45F1D009F57D
:104C140080394D45EDD0A9F58019E7E700245FE719
:104C2400CC685DE7CC6808345AE7CC680C3457E7A5
:104C3400042455E70025A4E70125A2E70225A0E7FF
:104C440003259EE704259CE7001002400004014070
:104C540000080140001C0140000021100000111058
:104C6400000031100AB1016170470904FBE7C36811
:104C74000B4214BF41610161704700002DE9F3410B
:104C8400054608B901203CE00368DB0710D42B6813
:104C94009F075DD42B68190700F194802B685A078D
:104CA40000F1BE80E869002840F02C81002028E053
:104CB4008F4C636803F00C03042B07D0636803F084
:104CC4000C03082B09D16368DE0306D523689C0313
:104CD400DDD56B68002BDAD1D4E76B68B3F5803F80
:104CE40012D1236843F480332360FFF7DBFA0646CE
:104CF40023689803CBD4FFF7D5FA801B6428F7D92F
:104D0400032002B0BDE8F0819BB9236823F480330B
:104D14002360236823F480232360FFF7C3FA064645
:104D240023689903B3D5FFF7BDFA801B6428F7D92C
:104D3400E6E7B3F5A02F236803D143F4802323606F
:104D4400CFE723F480332360236823F48023CBE765
:104D5400674C636813F00C0F07D0636803F00C030F
:104D6400082B10D16368DA030DD423689B0702D59E
:104D74002B69012B86D123686A6923F0F80343EA7F
:104D8400C203236086E72A695A4B6AB101221A607A
:104D9400FFF788FA064623689F07ECD4FFF782FAE8
:104DA400801B0228F7D9ABE71A60FFF77BFA0646A7
:104DB400236898077FF56EAFFFF774FA801B02280B
:104DC400F6D99DE7AA694A4C4B4BDAB101221A6025
:104DD400FFF768FA0646636A9B070DD54FF4FA524B
:104DE400464B1B68B3FBF2F3019300BF019B5A1EB1
:104DF4000192002BF9D151E7FFF754FA801B0228E6
:104E0400E9D97DE71A60FFF74DFA0646636A9F0702
:104E14007FF544AFFFF746FA801B0228F6D96FE707
:104E2400334CE369D80024D40127E36943F0805369
:104E3400E361E36903F080530093009B304E3368D1
:104E4400D90518D5EB68012B26D1236A43F0010359
:104E54002362FFF727FA41F288368046236A9B07CC
:104E64003FD5002F3FF41EAFE36923F08053E36185
:104E740018E70027E2E7336843F480733360FFF7F1
:104E840011FA80463368DA05DCD4FFF70BFAA0EB9D
:104E940008006428F6D933E7ABB9236A41F28838AD
:104EA40023F001032362236A23F004032362FFF740
:104EB400F9F90646236A9807D3D5FFF7F3F9801B5F
:104EC4004045F7D91CE7052B236A03D143F00403BB
:104ED4002362BAE723F001032362236A23F0040365
:104EE400B6E7FFF7DFF9A0EB0800B042B6D907E751
:104EF40000100240000042428004424208020020A6
:104F0400007000402A4B5A681C4602F00C02082A22
:104F14003DD00023274E022833602BD1FFF7C2F97E
:104F24000746236899011FD42B6AB3F5803F05D146
:104F34006268A96822F400320A436260696A62689E
:104F44000B4322F474121343636001233360FFF7AD
:104F5400A9F9054623689A013FF5A8AEFFF7A2F91F
:104F6400401B0228F6D9CBE6FFF79CF9C01B0228A8
:104F7400D7D9C5E6FFF796F9054623689B017FF567
:104F840095AEFFF78FF9401B0228F6D9B8E6012841
:104F94003FF4B7AE58682B6A00F480329A427FF42B
:104FA40071AE6B6A00F47010C01A18BF0120A8E635
:104FB400001002406000424230B5194B87B002AC89
:104FC40003F11005224618685968083303C2AB423E
:104FD4001446F7D101238DF80430022311498DF8CA
:104FE40005304B6803F00C02082A17D1C3F383423F
:104FF40006A80244DB0312F8102C0CD54B680A48AF
:10500400C3F34043504306AA134413F8143CB0FBC3
:10501400F3F007B030BD05485043FAE70248F8E71B
:10502400CC7600080010024000127A0000093D000E
:105034002DE9F0410D46044610B90120BDE8F08188
:10504400454A136803F007038B4229D321688E076E
:1050540031D4CA0744D4404A136803F007039D427D
:1050640067D322683D4D12F0040F6ED1130706D5A5
:105074006B68226923F4605343EAC2036B60FFF751
:105084009BFF6B68364AC3F30313D35CD840354B9C
:105094001860354B1868FFF7C3F80020BDE8F081AD
:1050A400136823F007030B431360136803F007032B
:1050B4009942C2D1CAE7294B11F0040F1EBF5A68A6
:1050C40042F4E0625A60080742BF5A6842F46052F0
:1050D4005A605A68A06822F0F00202435A60B8E7A6
:1050E40062681E4E012A33681BD113F4003FA4D01A
:1050F400736841F2883823F0030313437360FFF7A6
:10510400D1F807467368626803F00C03B3EB820FAF
:10511400A1D0FFF7C7F8C01B4045F3D90320BDE871
:10512400F081022A02D113F0007FE0E713F0020FAE
:10513400DDE7136823F007032B431360136803F0C0
:1051440007039D427FF479AF8BE76B68E16823F432
:10515400E0630B436B6089E70020024000100240CB
:10516400797700080802002004000020044B054A57
:105174005B68C3F30223D35C034A1068D8407047CA
:10518400001002408977000808020020044B054AF9
:105194005B68C3F3C223D35C034A1068D8407047EA
:1051A40000100240897700080802002003682DE9F6
:1051B400F341D907054620D5354CE369DA0032D4EA
:1051C4000127E36943F08053E361E36903F080530B
:1051D4000193019B2F4E3368DB0526D5236A13F414
:1051E400407336D1236A6A6823F4407313432362FD
:1051F4001FB1E36923F08053E3612868830706D570
:10520400234AA968536823F440430B43536010F0C6
:1052140010001BD01E4A69695368002023F48003E0
:105224000B43536012E00027D4E7336843F48073E0
:105234003360FFF737F880463368D805CED4FFF7DC
:1052440031F8A0EB08006428F6D9032002B0BDE8C9
:10525400F0816A6802F440729342C3D001200E4A7E
:10526400236A1060002023F4407110602162D90782
:10527400B8D5FFF717F841F288380646236A9A072B
:10528400B0D4FFF70FF8801B4045F7D9DDE700BF26
:1052940000100240007000404004424203680020B5
:1052A400DA6842F00102DA609A6802F00702062A1C
:1052B4001EBF1A6842F001021A60704770477047B7
:1052C40070477047036810B51A69044691070ED5F4
:1052D400DA6892070BD56FF002021A6101229B690A
:1052E40002779B0777D0FFF7EAFF00232377236831
:1052F4001A69500710D5DA6851070DD56FF004020A
:105304001A6102229B69227713F4407F204668D0F9
:10531400FFF7D5FF0023237723681A6912070FD5F7
:10532400DA6810070CD56FF008021A610422DB69F1
:105334002277990720465AD0FFF7C1FF002323772D
:1053440023681A69D20610D5DA68D0060DD56FF035
:1053540010021A610822DB69227713F4407F204689
:105364004BD0FFF7ACFF0023237723681A69D107DA
:1053740008D5DA68D20705D56FF0010220461A6114
:1053840000F0F6FB23681A69100608D5DA681106DE
:1053940005D56FF0800220461A6100F0BAF8236840
:1053A4001A69520608D5DA68500605D56FF040022E
:1053B40020461A61FFF785FF23681A69910622D5F2
:1053C400DA6892061FD56FF020022046BDE810402F
:1053D4001A6100F09DB8FFF771FF2046FFF770FFD8
:1053E40083E7FFF76BFF2046FFF76AFF92E7FFF7BB
:1053F40065FF2046FFF764FFA0E7FFF75FFF204645
:10540400FFF75EFFAFE710BD244A0368904212D055
:1054140002F5006290420ED0B0F1804F0BD0A2F59D
:105424009832904207D002F58062904203D002F590
:10543400806290421DD14A6823F070031343174AD7
:10544400904212D002F5006290420ED0B0F1804F2B
:105454000BD0A2F59832904207D002F580629042B8
:1054640003D002F58062904203D1CA6823F44073EA
:1054740013434A6923F08003134303608B68C362B8
:105484000B688362054B984203D003F5006398428E
:1054940001D10B690363012343617047002C014070
:1054A40010B50446A0B190F83D3003F0FF021BB9DB
:1054B40080F83C2000F024FE0223206884F83D306C
:1054C400211DFFF7A1FF0123002084F83D3010BD0A
:1054D400012010BD90F83C3030B5012B4FF0020391
:1054E40014D0046880F83D306268A3680D68496888
:1054F40022F0700223F080030B432A436260A3600E
:10550400012380F83D30002380F83C30184630BD3C
:10551400704770470368DA6822F49072DA605A6957
:1055240022F001025A61202380F83A3070470000CB
:1055340038B505460368C1681A69192422F4405233
:105544000A431A6182680069D9680243686921F4D0
:10555400B05121F00C0102430A43DA605A69A96987
:1055640022F440720A435A610D4A934214D1FFF760
:105574000DFE60436C686422A400B0FBF4F0B0FB41
:10558400F2F402FB14031B013233B3FBF2F3296878
:1055940003EB04138B6038BDFFF7E8FDE9E700BFB8
:1055A40000380140F8B504460E4617461D462168EA
:1055B4000B6836EA030301D10020F8BD6B1CF7D059
:1055C40095B923680320DA6822F4D072DA605A6944
:1055D40022F001025A61202384F8393084F83A30E9
:1055E400002384F83830F8BDFEF75CFEC01B85420A
:1055F400DDD2E6E710B5044640B390F8393003F045
:10560400FF021BB980F8382000F08EFD24232268A5
:1056140084F83930D368204623F40053D360FFF76D
:1056240087FF236800201A6922F490421A615A699C
:1056340022F02A025A61DA6842F40052DA60202326
:10564400E06384F8393084F83A3010BD012010BD8D
:105654002DE9F0411F4690F839300446202B0D46C1
:1056640090464ED1002949D0002A47D090F83830CE
:10567400012B46D0012380F838300023C363212353
:1056840080F83930FEF70EFE0646A4F82480A4F80C
:105694002680E38C9BB26BB93B46324640212046C0
:1056A400FFF780FFA8B9202384F8380084F8393044
:1056B400BDE8F081E38C3246013B9BB2E384A368EE
:1056C4008021B3F5805F20463B460ED1FFF76AFF89
:1056D40010B10320BDE8F0812B882268C3F30803CE
:1056E4005360236943B90235D3E7FFF75BFF002812
:1056F400EFD123682A785A600135CAE70120BDE852
:10570400F0810220BDE8F08138B50446134694F8D0
:105714003920202A2AD139B333B394F83820012A06
:1057240024D00122002584F838202122E384206B30
:10573400E56384F839200E4AA384216282620D4A0B
:105744004563C2620C4A026322680432FFF716F80A
:105754006FF04002236828461A605A6984F838506A
:1057640042F080025A6138BD012038BD022038BDA4
:1057740013580008415800080D590008134690F8C2
:105784003A2073B5202A054638D1002934D0002B9D
:1057940032D090F83820012A30D00122002480F839
:1057A4003820222281628385C46380F83A20406BCA
:1057B400134A2E688262134A4463C262124A026325
:1057C4000A46311DFEF7DAFF20462B6801941A6859
:1057D40001925A6885F838400192019ADA6842F4D5
:1057E4008072DA605A6942F001025A615A6942F0E1
:1057F40040025A6102B070BD0120FBE70220F9E7C4
:105804004B580008015900080D590008704708B5A5
:105814000368426A1B6813F020030AD1D384136817
:105824005A6922F080025A61DA6842F04002DA6072
:1058340008BD1046FFF7EAFF08BD704708B5406A87
:10584400FFF7FBFF08BD08B50368426A1B6813F045
:10585400200310D1D3851368D96821F48071D960ED
:10586400596921F001015961596921F040015961D7
:10587400202382F83A30104600F01AFE08BD90F852
:105884003A3010B5222B36D183680169B3F5805FB5
:105894000268836A23D15268E9B9C2F3080223F883
:1058A400022B8362C48D013CA4B2C4858CB9036805
:1058B400DA6822F02002DA60DA6822F48072DA60B0
:1058C4005A6922F001025A61202380F83A3000F02C
:1058D400EFFD002010BDD2B223F8012BE1E721B97E
:1058E400591C526881621A70DCE75268591C816243
:1058F40002F07F02F7E7022010BD704708B5406A46
:10590400FFF7FBFF08BD7047416A08B50B685A6989
:1059140091F8390021280AD1120608D50022CA8438
:10592400DA6822F0C002DA60202281F839205B694B
:1059340091F83A20222A06D15B0604D500230846B2
:10594400CB85FFF7E7FDCB6B084643F01003CB6331
:10595400FFF7D9FF08BD0000036870B51A68044654
:105964001607D9685D6907D196065AD58D0658D5AC
:10597400BDE87040FFF783BF15F0010502D111F4B3
:10598400907F4ED0D30705D5CE0542BFE36B43F0DD
:105994000103E363500704D51DB1E36B43F0020335
:1059A400E363930704D51DB1E36B43F00403E3639E
:1059B400160704D51DB1E36B43F00803E363E36BFF
:1059C400002B66D0950604D5880602D52046FFF73D
:1059D40056FF236820465D69E26B110702D415F077
:1059E40040051AD0FFF796FD23685A69520610D570
:1059F4005A69606B22F040025A6150B1254B4363EF
:105A0400FEF7FAFE002844D0606BBDE87040436B9B
:105A140018472046FFF777FF70BDFFF774FFE56373
:105A240070BD160627D50D0625D594F83920212AF0
:105A34002FD1A268B2F5805F226A17D11188C1F311
:105A440008015960216979B902322262E28C013A73
:105A540092B2E284EAB9DA6822F08002DA60DA68A3
:105A640042F04002DA6070BD0132EEE7511C21625F
:105A740012785A60EAE750060BD54A0609D5DA6867
:105A8400204622F04002DA60202384F83930FFF700
:105A9400BDFE70BD9D5A000808B50023406AC38549
:105AA400C384FFF730FF08BD002310B50F4CC900B5
:105AB40007290FDC61B141F2210213F4004F4FEAD0
:105AC40043039BB201F1FF3118BF53400029F4D1C5
:105AD400184610BD10F8012B083982EA132234F855
:105AE400122082EA03239BB2E2E700BF08000020F1
:105AF400174B10B51A78174C12B12278032A10D814
:105B040001221A702378032B0BD8DFE803F0020B71
:105B14000E110D21104800F0FBFC23780133DBB299
:105B2400237010BD0D210D48F5E71D210C48F2E747
:105B340015210C4800F0ECFC0520FEF7B9FB0A2106
:105B4400094800F0E5FC094800F0CAFDE5E700BF9C
:105B54008C0200208D020020E7760008F57600080C
:105B64000377000821770008377700084277000898
:105B74000268084B9A420BD1074A13680133136039
:105B8400064A136801331360054A1368013313602E
:105B9400704700BF001000409802002094020020CB
:105BA4009002002010B514460A230248FFF750FD66
:105BB400204610BD4C04002010B596B028220021C8
:105BC4000CA800F0FDFC1422002101A800F0F8FC50
:105BD400182200210DEB020000F0F2FC01231093C7
:105BE4001023022411934FF460130CA815930C9402
:105BF4001394FFF743F80F234FF4806201930023BB
:105C0400214601A80393049205930294FFF710FA26
:105C14004FF4004306A806940893FFF7C7FA16B09A
:105C240010BD000080B5BA4A8CB05168106805AB4D
:105C340003C31189927AB74D19809A70FEF714FB49
:105C4400FFF7BAFF1022002108A800F0B9FCAB69E5
:105C5400002243F01003AB61AB6949F2400103F049
:105C640010030193019BAB69AB4843F00403AB61A0
:105C7400AB69002403F004030293029BAB69012681
:105C840043F00803AB61AB69022703F008030393F5
:105C9400039BAB694FF0090843F02003AB61AB6988
:105CA4004FF00B0903F020030493049BFEF7DAFF83
:105CB40000224EF2F2019948FEF7D4FF002248F286
:105CC400D8019748FEF7CEFF002204219548FEF73D
:105CD400C9FF49F2400308A98F48089309960A941A
:105CE4000B97FEF7D3FE4EF2F20308A98B480893F4
:105CF40009960A940B97FEF7C9FE48F2D80308A93F
:105D04008748089309960A940B97FEF7BFFE04236D
:105D14000B974FF4602708A98248089309960A94C0
:105D2400FEF7B4FE6B694FF4E13A33436B616B6980
:105D34007D4D33400093009B7C4B28462B60AC6028
:105D44002C732C75EF616C602E61089409940A948D
:105D5400FEF7DEFB08A92846754DCDF8208009968C
:105D64000A94FEF72FFB734B28462B60AC602C7310
:105D74002C75EF616C602E61089409940A94FEF707
:105D8400C7FB0A2308A928466B4D089309960A9471
:105D9400FEF718FB694B28462B60AC602C732C75FE
:105DA400EF616C602E61089409940A94FEF7B0FBCD
:105DB40008A9284609960A94CDF82090FEF702FB1C
:105DC40041F6FF035E4F5F4AC7F80C804FF00C08A2
:105DD40038465D4E87E80C0008940994BC60BC61A9
:105DE400FFF75EFB08A9384608940994FFF772FB95
:105DF400564B574D304686E80804B460F46034616D
:105E0400B461F461C6F81480FFF7F4FB514B2846E3
:105E140085E80804AC60EC602C61AC61EC61C5F809
:105E24001480FFF7E7FB4C4B4C4880E8080484607F
:105E3400C46004618461C461C0F81480FFF7DAFBB4
:105E4400224621461020FEF701FC1020FEF732FC0A
:105E5400224621460F20FEF7F9FB0F20FEF72AFC0D
:105E6400224621460E20FEF7F1FB0E20FEF722FC0F
:105E7400224621461120FEF7E9FB1120FEF71AFC09
:105E8400224621462F20FEF7E1FB2F20FEF712FCCD
:105E9400224621463420FEF7D9FB3420FEF70AFCC3
:105EA400224621463620FEF7D1FB3620FEF702FCBF
:105EB400224621461220FEF7C9FB1220FEF7FAFB08
:105EC400224621462520FEF7C1FB2520FEF7F2FBE2
:105ED400224621462620FEF7B9FB2620FEF7EAFBE0
:105EE4003846FFF7DBF91E4B21461B681D4C9868AA
:105EF40000F0FEFB1C4800F0F3FB494605A8FFF741
:105F0400D3FD0146194800F063FB304630E000BF82
:105F1400DC76000800100240001001400008014037
:105F2400000C0140001401406403002000240140DF
:105F3400F00200200028014094030020003C0140AE
:105F44008C040020001000404C0400200038014064
:105F54000C05002000440040004C0040CC0400200C
:105F64000C0200209402002059770008667700088C
:105F7400164900F067FA2846154900F063FA154EF1
:105F8400154D2368642B05D902213046FEF76FFEB8
:105F9400002323602B68B3F57A7F03D9FFF7A8FDAC
:105FA40000232B60094FDFF83480BB68002B09DC29
:105FB400074FDFF82C80BB68002BE2DD404600F081
:105FC40059FAF8E7404600F055FAEEE74C05002090
:105FD4005809002000080140900200204C040020D1
:105FE4000C050020704700000E4B82B09A6942F005
:105FF40001029A619A6902F001020092009ADA6938
:1060040042F08052DA61DB69074A03F0805301935E
:10601400019B536823F0E06343F08063536002B054
:10602400704700BF001002400000014010B5044654
:106034008AB01022002106A800F0C2FA23682A4A76
:1060440093421CD1294B2A489A6906A942F400724A
:106054009A619A6902F400720092009A9A6942F075
:1060640008029A619B6903F008030193019B0223D0
:10607400069303230793FEF709FD0AB010BD1D4ADA
:10608400934219D1194B9A6942F480629A619A69D0
:1060940002F480620292029A9A6942F010029A61B2
:1060A4009B6903F010030393039B012306930323CB
:1060B40006A907931048DEE7104A9342DDD10B4B43
:1060C4009A6942F400429A619A6902F40042049285
:1060D400049A9A6942F010029A619B6903F01003D2
:1060E4000593059B0223E1E70024014000100240D0
:1060F400000C01400028014000100140003C014018
:106104000268084B82B09A420AD103F50033DA6977
:1061140042F01002DA61DB6903F010030193019B82
:1061240002B070470010004070B505468AB01022D6
:10613400002106A800F044FA2B68604A934229D152
:106144005F4B06A9DA695F4842F40022DA61DA6932
:1061540002F400220092009A9A6942F010029A61B5
:106164009B6903F010030193019B4FF48063069332
:106174000223079303230993FEF788FC4FF400637B
:106184000693002306A94F4807930893FEF77EFC65
:106194000AB070BD4C4A934250D1494B06A99A6942
:1061A4004A4842F480429A619A69002602F4804285
:1061B4000292029A9A69464C42F004029A619B69DF
:1061C40003F004030393039B4FF400730693022329
:1061D400079303230993FEF759FC4FF480633B486C
:1061E40006A9069307960896FEF750FC394B2046FD
:1061F40084E848008023A660E36026616661A661A6
:10620400E661FEF77BFA08B1FFF7ECFE6C636562AA
:10621400314B324C23601023802263600023E26000
:10622400A36023616361A361E3612046FEF766FA1C
:1062340008B1FFF7D7FE2C636562A9E7284A9342A9
:10624400A6D11F4B06A9DA69204842F40032DA616C
:10625400DA69002602F400320492049A9A69214C05
:1062640042F004029A619B6903F004030593059BC1
:10627400042306930223079303230993FEF706FCE2
:106284000823124806A9069307960896FEF7FEFB14
:10629400154B204684E848008023A660E36026610D
:1062A4006661A661E661FEF729FA08B1FFF79AFE76
:1062B4006C6365620D4B0E4CACE700BF004C0040B4
:1062C4000010024000100140003801400008014065
:1062D400C403002058000240440002402003002070
:1062E40000440040AC0200206C00024080000240E8
:1062F400080400207047FEE7FEE7FEE7FEE770476C
:1063040070477047FDF7C2BF0148FEF7E3BA00BF0C
:10631400200300200148FEF7DDBA00BFC4030020BB
:106324000148FEF7D7BA00BFAC0200200148FEF7CF
:10633400D1BA00BF0804002008B50448FDF7CCFF1B
:10634400BDE808400248FDF7C7BF00BF6403002052
:10635400F00200200148FFF7FFBA00BF4C04002000
:106364000148FFF7F9BA00BF0C0500200148FDF70A
:10637400B3BF00BF940300200148FFF7EDBA00BF8C
:10638400CC0400200148FEF79DBF00BF8C04002010
:1063940070B50E4615460C46A31B9D4201DC2846EB
:1063A40070BDAFF3008004F8010BF5E708B50A4BA4
:1063B4000246196809B9094919606946186802440E
:1063C4008A4206D900F0D2F80C2303604FF0FF3064
:1063D40008BD1A6008BD00BF9C020020680D0020A3
:1063E4004FF0FF3070474FF4005300204B6070476C
:1063F40001207047002070470E4B1A6842F00102DA
:106404001A6059680C4A0A405A601A6822F0847269
:1064140022F480321A601A6822F480221A605A68C0
:1064240022F4FE025A604FF41F029A60034A044B9E
:106434009A607047001002400000FFF80040000816
:1064440000ED00E0002330B40568074C4B600B609E
:106454008B600648064B012285420CBF2046184635
:1064640030BC0C31FFF78AB90C0500200044004011
:106474004C04002010B501680A4B0B4A0B4C9142A6
:1064840018BF1C4663682344187B00F0B9F863689E
:106494000133B3F5806FA8BF00236360A368013B99
:1064A400A36010BD4C0500200044004058090020A2
:1064B40038B50268114B124C9A42124B124D08BF68
:1064C4001C46124B08BF1D4623680133B3F5806F89
:1064D400A8BF00232360A3680133B3F5806FA360D2
:1064E40001DBFFF7C7FF236804F10C0119442846B8
:1064F400BDE838400122FFF741B900BF0044004025
:106504004C050020580900204C0400200C050020F4
:106514000A4601460148FFF7F7B800BF0C05002002
:10652400002103E00B4B5B58435004310A480B4BEA
:1065340042189A42F6D30A4A02E0002342F8043B86
:10654400084B9A42F9D3FFF757FF00F015F8FFF70D
:1065540069FB7047347800080000002070020020B6
:1065640070020020680D0020FEE70000014B18684F
:10657400704700BF0C02002070B500250C4E0D4C76
:10658400A41BA410A54209D101F092F800250A4EDB
:106594000A4CA41BA410A54205D170BD56F82530A1
:1065A40098470135EEE756F8253098470135F2E76C
:1065B4002C7800082C7800082C7800083078000823
:1065C40003460244934200D1704703F8011BF9E7E4
:1065D4000FB40A4B13B51C6824B1A36913B9204640
:1065E40000F0EEFA05AB049AA1682046019300F08E
:1065F400AFFC02B0BDE8104004B070470C020020AC
:1066040038B5084B05461C6824B1A36913B9204664
:1066140000F0D6FAA26829462046BDE8384000F0CA
:1066240045BF00BF0C02002070B50E46054618B1E8
:1066340083690BB900F0C4FAAB69AC6813B9284696
:1066440000F0BEFA234B9C4217D16C68A3891B0748
:106654001DD52369DBB1013EA36816F8011F013B78
:10666400A360E9B9002B2EDA22460A21284600F05D
:10667400F5F8013011D00A2070BD174B9C4201D1AE
:10668400AC68E3E7154B9C4208BFEC68DEE72146A3
:10669400284600F035F90028DDD04FF0FF3070BDFA
:1066A400002B04DAA269934206DB0A2904D023688A
:1066B4005A1C22601970CFE72246284600F0CEF813
:1066C4000130C9D1E9E70A2023685A1C22601870F6
:1066D40070BD00BFB8770008D87700089877000825
:1066E400024B01461868FFF79FBF00BF0C02002051
:1066F40000294FF480630CBF0222002200F000B88E
:106704002DE9F7431D46514B04461E680F4690463B
:1067140026B1B36913B9304600F052FA4C4B9C428F
:1067240052D17468B8F1020F06D0B8F1010F00F22B
:106734008980002DC0F286802146304600F0D6F9CB
:10674400616B41B104F14403994202D0304600F038
:106754002DFB002363630023A3616360A3891B06ED
:1067640003D52169304600F021FBA389B8F1020F5B
:1067740023F44A6323F00303A3815DD001AB6A468B
:106784002146304600F0A6FAA3891843A0812DBB08
:10679400009D284600F002FB074600284ED1DDF894
:1067A4000090A9453CD14FF0FF30A38943F0020388
:1067B400A3810023A36004F1470323602361012321
:1067C400636103B0BDE8F083224B9C4201D1B468FD
:1067D400A8E7214B9C4208BFF468A3E7002FD8D058
:1067E400B36913B9304600F0EBF9B8F1010F08BFF3
:1067F400A389276004BF43F00103A381A389276110
:1068040013F0080065611BD013F001004FF0000382
:106814001FBF6D42A360A561184608BFA560D0E7FD
:10682400484600F0BBFA07460028BCD0A3894D4671
:1068340043F08003A381D3E70020B6E7A946F5E738
:10684400A060BEE74FF0FF30BBE700BF0C020020A2
:10685400B8770008D877000898770008F8B50E468E
:106864001446054618B183690BB900F0A9F9214B08
:106874009C422AD16C68A369A360A3891A072ED508
:10688400236963B323692068F6B2C01A6369374683
:10689400984204DB2146284600F028F928BBA36867
:1068A4000130013BA36023685A1C22601E70636997
:1068B400984204D0A389DB0719D50A2E17D12146A3
:1068C400284600F013F990B10FE00B4B9C4201D124
:1068D400AC68D0E7094B9C4208BFEC68CBE7214683
:1068E400284600F00DF80028CCD04FF0FF3738468A
:1068F400F8BD00BFB8770008D8770008987700087B
:10690400324B70B51D6806460C4625B1AB6913B908
:10691400284600F055F92E4B9C420FD16C68B4F90F
:106924000C309AB215072CD4D00611D40922326047
:1069340043F04003A3814FF0FF3070BD254B9C42D0
:1069440001D1AC68EBE7244B9C4208BFEC68E6E756
:10695400510712D5616B41B104F14403994202D04D
:10696400304600F023FA00236363A38923F0240351
:10697400A3810023636023692360A38943F0080390
:10698400A38123694BB9A38903F42073B3F5007F72
:1069940003D02146304600F0C1F9A28912F0010368
:1069A4000CD00023A36063695B42A361236953B9DC
:1069B400B4F90C3013F08000BAD170BD920758BFFF
:1069C4006369A360F2E70020F7E700BF0C02002030
:1069D400B8770008D8770008987700088A892DE9E5
:1069E400F041054610070C465AD44B68002B05DCD1
:1069F4000B6C002B02DC0020BDE8F081E66A002E5F
:106A0400F9D0002312F480522F682B6033D0606DCC
:106A1400A3895A0705D56368C01A636B0BB1236C4D
:106A2400C01A00230246E66A216A2846B047431C7E
:106A3400A38906D129681D294BD82B4ACA40D607F9
:106A440047D5002262602269D904226004D5421C21
:106A540001D12B6803B96065616B2F600029CAD02E
:106A640004F14403994202D0284600F09FF9002023
:106A74006063BDE8F081216A01232846B047411CC8
:106A8400C6D12B68002BC3D01D2B01D0162B01D1EE
:106A94002F60B0E7A38943F04003A381BDE8F081F0
:106AA4000F69002FA7D0930718BF00230E6808BFF3
:106AB4004B69A6EB07080F608B60B8F1000F9ADDF5
:106AC40043463A46216A2846A66AB047002807DCAE
:106AD400A38943F04003A3814FF0FF30BDE8F08168
:106AE4000744A8EB0008E8E70100402038B50B692B
:106AF40005460C46DBB118B183690BB900F060F8A8
:106B04000C4B9C4209D16C68B4F90C307BB1214622
:106B14002846BDE83840FFF761BF074B9C4201D1CE
:106B2400AC68F1E7054B9C4208BFEC68ECE7002039
:106B340038BD00BFB8770008D877000898770008F8
:106B4400014900F0A9B800BFF16A0008002310B59C
:106B5400044603604360836081814366C2810361AC
:106B640043618361194608225C30FFF729FD054B18
:106B740024626362044BA362044BE362044B236309
:106B840010BD00BF3D7500085F75000897750008CB
:106B9400BB75000870B568254A1E55430E4605F1BD
:106BA400740100F04FF9044640B1002180E842002E
:106BB4000C30A06005F16802FFF702FD204670BDAD
:106BC400836910B5044633BB8364C3640365124B05
:106BD400124A1B688262984204BF0123836100F059
:106BE4001FF86060204600F01BF8A060204600F00B
:106BF40017F80022E06004216068FFF7A7FF012274
:106C04000921A068FFF7A2FF02221221E068FFF722
:106C14009DFF0123A36110BD94770008456B000814
:106C2400F8B51C4B07461E68B36913B93046FFF725
:106C3400C7FF4836B4687368013B03D5336833B182
:106C44003668F7E7B4F90C506DB16834F4E7042101
:106C54003846FFF79FFF30600028F1D10C2304462B
:106C64003B602046F8BD4FF6FF73E3810123656660
:106C7400A3812560A560656025616561A561082221
:106C8400294604F15C00FFF79BFC6563A563A564DA
:106C9400E564E6E7947700082DE9F84380468946E1
:106CA400002600F1480414B93046BDE8F883A5680D
:106CB4006768013F01D52468F5E7AB89012B07D943
:106CC400B5F90E30013303D029464046C847064380
:106CD4006835EEE770B50E46B1F90E1090B0002994
:106CE40014461D4607DA00232B60B3891A0610D414
:106CF4004FF480630EE001AA00F084FC0028F2DB6C
:106D0400029A02F47042A2F500535A425A412A6090
:106D1400EEE740230020236010B070BD8B8973B56B
:106D24009D0706460C4607D504F1470323602361FB
:106D34000123636102B070BD01AB6A46FFF7CAFF6D
:106D440000990546304600F07DF848B9B4F90C3096
:106D54009A05EFD423F0030343F00203A381E3E78E
:106D64000D4BB362A389206043F08003A381009B91
:106D740020616361019B5BB1B4F90E10304600F0F1
:106D840053FC28B1A38923F0030343F00103A38137
:106D9400A3891D43A581CDE7456B0008024B01463D
:106DA400186800F04FB800BF0C02002038B5054643
:106DB400002943D051F8043C0C1F002BB8BFE41841
:106DC40000F062FC1E4A1368104633B96360146015
:106DD4002846BDE8384000F058BCA3420BD92168CE
:106DE4006218934201BF1A685B685218226063609C
:106DF4000460EDE713465A680AB1A242FAD9196849
:106E04005818A0420BD120680144581882421960D6
:106E1400DED110685268014419605A60D8E702D97B
:106E24000C232B60D4E7206821188A4201BF116823
:106E340052680918216062605C60C9E738BD00BF10
:106E4400A002002070B5CD1C25F0030508350C2DDB
:106E540038BF0C25002D064601DBA94203D90C23BB
:106E64003360002070BD00F00FFC234A14682146F3
:106E740091B9224C23681BB9304600F04DFB2060C9
:106E84002946304600F048FB431C26D10C233046EB
:106E9400336000F0FAFBE4E70B685B1B1AD40B2B9E
:106EA4000FD90B60CC18CD50304600F0EEFB04F146
:106EB4000B00231D20F00700C31A1BD05A42E250D6
:106EC40070BD8C420BBF63684B681360636018BF6E
:106ED4000C46E9E70C464968CAE7C41C24F00304DD
:106EE400A04205D0211A304600F016FB0130CDD067
:106EF4002560D9E770BD00BFA0020020A4020020D5
:106F0400936810B4013B002B936008DA9469A342A0
:106F140002DBCBB20A2B02D110BCFFF79FBC136873
:106F2400581C10601970C8B210BC7047F8B50646FA
:106F34000F461446D518AC4201D1002007E03A466A
:106F440014F8011B3046FFF7DBFF431CF3D1F8BDF7
:106F54002DE9F04F9DB00C4617460393064618B131
:106F640083690BB9FFF72CFE7C4B9C4257D17468A4
:106F7400A38918075DD52369002B5AD000230993F0
:106F840020238DF8293030234FF0010B8DF82A305F
:106F9400B846454615F8013B002B55D1B8EB070A16
:106FA4000BD053463A4621463046FFF7BFFF013027
:106FB40000F0C480099B5344099398F80030002BD7
:106FC40000F0BC8000234FF0FF3204930793059236
:106FD40006938DF853301A9305222978604800F0FF
:106FE40045FB05F10108049B002831D1D90644BFB3
:106FF40020228DF853201A0744BF2B228DF85320EA
:107004002A782A2A2CD000210A20079AA84698F820
:1070140000300135303B092B6DD971B326E0514B5B
:107024009C4201D1B468A3E74F4B9C4208BFF4686B
:107034009EE721463046FFF763FC00289ED04FF0C0
:10704400FF301DB0BDE8F08F252BA7D0A846A0E7E0
:10705400434A4546801A0BFA00F018430490BBE7F4
:10706400039A111D12680391002A01DB079204E0C0
:10707400524243F002030792049398F800302E2BF7
:1070840010D198F8013008F101012A2B37D1039B64
:1070940008F102081A1D1B680392002BB8BF4FF0B9
:1070A400FF330593314D032298F80010284600F071
:1070B400DDFA40B14023401B03FA00F0049B08F1C1
:1070C40001080343049398F800100622284808F1A5
:1070D40001078DF8281000F0C9FA002834D0254B98
:1070E40003BB039B073323F0070308330393099B74
:1070F4004B4409934CE700FB0232012186E700234D
:107104000A2518460593884698F800200131303A3C
:10711400092A03D9002BC5D00590C3E705FB00203D
:107124000123F0E703AB00932246134B04A9304636
:10713400AFF30080B0F1FF3F8146D8D1A3895B064D
:107144003FF57DAF09987CE703AB009322460A4BD9
:1071540004A9304600F08AF8ECE700BFB8770008CD
:10716400F8770008D877000898770008FE770008B9
:107174000278000800000000316F00082DE9F04794
:1071840091461F468A680B6906469342B8BF134668
:10719400C9F8003091F843200C46DDF8208012B184
:1071A4000133C9F800302368990642BFD9F800308A
:1071B4000233C9F80030256815F0060507D104F13B
:1071C400190AE368D9F800209B1A9D422ADB94F837
:1071D40043302268003318BF012392062FD404F1F0
:1071E400430239463046C047013022D02368E5685F
:1071F40003F00603042B18BF0025D9F800204FF034
:10720400000908BFAD1AA368226908BF25EAE5751D
:107214009342C4BF9B1AED181A344D451BD100206C
:10722400BDE8F0870123524639463046C047013055
:1072340003D14FF0FF30BDE8F0870135C1E73020BE
:10724400E11881F843005A1C94F845102244023393
:1072540082F84310C3E70123224639463046C0472B
:107264000130E6D009F10109D7E700002DE9F04328
:1072740017460A7E85B06E2A984606460C460C9B35
:1072840001F1430E00F0BC801AD8632A2ED00AD82C
:10729400002A00F0C880582A00F08A8004F14205D0
:1072A40084F842202AE0642A01D0692AF6D12168B0
:1072B4001A6811F0800F23D0111D1960136827E09C
:1072C400732A00F0B48008D86F2A2AD0702AE5D136
:1072D4000A6842F020020A6003E0752A21D0782A65
:1072E400DCD178226F4984F8452064E01A6801F102
:1072F4004205111D1960136884F842300123A3E08C
:1073040011F0400F02F104011960D7D0B2F9003036
:10731400002B03DA2D225B4284F8432062490A22BF
:1073240017E02068196810F0800F03D0081D18605A
:107334000B6806E010F0400F01F104001860F7D06C
:107344000B886F2A14BF0A2208225749002084F8A8
:1073540043006568002DA560C0F29C80206820F081
:1073640004002060002B3FD1002D40F0958075462D
:10737400082A0BD12368DA0708D5236962689A4280
:10738400DEBF302305F8013C05F1FF35AEEB050304
:107394002361CDF800803B4603AA21463046FFF71F
:1073A400EDFE013055D14FF0FF3005B0BDE8F0835C
:1073B40081F845203C492268186812F0800F00F1DA
:1073C40004051D6001D0036802E05506FBD503885F
:1073D400D00744BF42F0200222601BB9226822F089
:1073E400200222601022B1E77546B3FBF2F002FBE3
:1073F4001033CB5C05F8013D03460028F5D1B7E70F
:1074040008681A6810F0800F496904D0101D1860CC
:107414001368196007E010F0400F02F104001860CF
:107424001368F6D01980002375462361B1E71A6802
:10743400111D1960156800216268284600F016F9CC
:1074440008B1401B606063682361002384F8433003
:107454009FE723692A4639463046C0470130A2D007
:1074640023689B0707D5002504F11909E368039AEB
:107474009B1A9D4205DBE068039B9842B8BF1846FF
:1074840093E701234A4639463046C04701308AD043
:107494000135EBE7002BA7D10B7804F1420584F802
:1074A400423065E71A7800080978000870B50D467F
:1074B4001446064618B183690BB9FFF781FB134BD9
:1074C4009C4212D17468A368013B002BA36016DAB6
:1074D400A269934202DBEBB20A2B10D12246294661
:1074E4003046BDE87040FFF7B9B9094B9C4201D161
:1074F400B468E8E7074B9C4208BFF468E3E72368F5
:10750400E8B25A1C22601D7070BD00BFB877000835
:10751400D87700089877000838B50023054C05464D
:1075240008462360FEF742FF431C02D1236803B1DF
:107534002B6038BD640D002010B50C46B1F90E1057
:1075440000F0A4F80028ABBF636DA3891B1823F4D3
:107554008053ACBF6365A38110BD2DE9F0411F4684
:107564008B890546DB050C46164605D50223002209
:10757400B1F90E1000F068F8A389324623F4805361
:10758400A381B4F90E103B462846BDE8F04100F053
:1075940017B810B50C46B1F90E1000F055F8431C9D
:1075A400A38915BF606523F4805343F48053A381FA
:1075B40018BFA38110BDB1F90E1000F013B800007C
:1075C40038B50546084611460022054C22601A4685
:1075D400FEF7E8FA431C02D1236803B12B6038BDDF
:1075E400640D002038B50023054C05460846236089
:1075F400FEF7F6FE431C02D1236803B12B6038BDAD
:10760400640D002038B50023064C05460846114693
:107614002360FEF7E8FE431C02D1236803B12B600C
:1076240038BD00BF640D002038B50023054C054665
:1076340008462360FEF7DCFE431C02D1236803B135
:107644002B6038BD640D002038B505460846114648
:107654000022054C22601A46FEF7CCFE431C02D1E0
:10766400236803B12B6038BD640D002010B5C9B286
:1076740002449042034601D1002010BD1C78013021
:107684008C42F6D1184610BD7047704738B5054690
:10769400084611460022054C22601A46FEF778FE81
:1076A400431C02D1236803B12B6038BD640D002054
:1076B400F8B500BFF8BC08BC9E467047F8B500BFDB
:0876C400F8BC08BC9E467047AB
:1076CC0002030405060708090A0B0C0D0E0F101017
:1076DC00000102030405060708090A41542B43570D
:1076EC004D4F44453D330D0A0041542B4349504DF9
:1076FC0055583D310D0A0041542B43575341503DD1
:10770C0022424C55455F54455354222C22222C3591
:10771C002C300D0A0041542B4349505345525645C9
:10772C00523D312C343030300D0A0041542B43493A
:10773C004653520D0A004553502053657474696EBC
:10774C006720436F6D706C657465200D0055617218
:10775C0074205374617274200D004372632067654A
:10776C006E6572617465202578200D0A000000009A
:10777C0000000000000102030406070809000000D5
:10778C0000010203040000001002002000000000B1
:10779C0000000000000000000000000000000000DD
:1077AC0000000000000000000000000000000000CD
:1077BC0000000000000000000000000000000000BD
:1077CC0000000000000000000000000000000000AD
:1077DC00000000000000000000000000000000009D
:1077EC00000000000000000000000000232D302BE2
:1077FC002000686C4C0065666745464700303132A6
:10780C0033343536373839414243444546003031FC
:10781C00323334353637383961626364656600005B
:04782C000942000805
:04783000E541000826
:10783400010000001000000000002110422063300D
:107844008440A550C660E770088129914AA16BB1B4
:107854008CC1ADD1CEE1EFF131121002733252225C
:10786400B5529442F772D662399318837BB35AA304
:10787400BDD39CC3FFF3DEE362244334200401142C
:10788400E664C774A44485546AA54BB52885099554
:10789400EEE5CFF5ACC58DD55336722611163006FC
:1078A400D776F6669556B4465BB77AA719973887A4
:1078B400DFF7FEE79DD7BCC7C448E5588668A778BC
:1078C4004008611802282338CCC9EDD98EE9AFF9F4
:1078D400488969990AA92BB9F55AD44AB77A966A9C
:1078E400711A500A333A122AFDDBDCCBBFFB9EEB44
:1078F400799B588B3BBB1AABA66C877CE44CC55C6C
:10790400222C033C600C411CAEED8FFDECCDCDDD93
:107914002AAD0BBD688D499D977EB66ED55EF44E3B
:10792400133E322E511E700E9FFFBEEFDDDFFCCFE3
:107934001BBF3AAF599F788F8891A981CAB1EBA137
:107944000CD12DC14EF16FE18010A100C230E320B3
:107954000450254046706760B9839893FBA3DAB35B
:107964003DC31CD37FE35EF3B1029012F322D23203
:107974003542145277625672EAB5CBA5A89589852B
:107984006EF54FE52CD50DC5E234C324A014810453
:107994006674476424540544DBA7FAB79987B897FB
:1079A4005FE77EF71DC73CD7D326F2369106B016A3
:1079B40057667676154634564CD96DC90EF92FE9BB
:1079C400C899E9898AB9ABA94458654806782768F3
:1079D400C018E1088238A3287DCB5CDB3FEB1EFB9B
:1079E400F98BD89BBBAB9ABB754A545A376A167A43
:1079F400F10AD01AB32A923A2EFD0FED6CDD4DCD6B
:107A0400AABD8BADE89DC98D267C076C645C454C92
:107A1400A23C832CE01CC10C1FEF3EFF5DCF7CDF3A
:107A24009BAFBABFD98FF89F176E367E554E745EE2
:107A3400932EB23ED10EF01E0024F400100200205A
:107A440000000000B8770008D8770008987700088D
:107A54000000000000000000000000000000000022
:107A64000000000000000000000000000000000012
:107A74000000000000000000000000000000000002
:107A840000000000000000000000000000000000F2
:107A940000000000000000000000000000000000E2
:040000050800652565
:00000001FF
